:200000000C94AF021895189518951895189518951895189518951895189518951895189519
:200020001895189518951895189518951895189518951895189518951895189518951895F0
:20004000189518950C94CA00189518951895189518951895000703060204000501070306A2
:2000600002050106020038183010200028083818301028083010001C0C1808100014041C04
:200080000C18081404180800E060C0408000A020E060C040A020C0400605040302302820F0
:2000A00018101814100C08C0A08060400E94D00022E008EA10E00E94610078940E94BD0183
:2000C000FDCFF801218322E0F8012083089506B7102F17FFFCCF01B1087F089503B904EC1D
:2000E00006BFF5DF0895BA93AA93D80104EC06BFEEDF003811F0003911F413B11C93A991C1
:20010000B99108950E94C6022801822F0091A900000F02B904EC06BFDADF003611F00836CD
:2001200079F4A0E001C0A395A81750F4B0E082010A0F1B1FD8DF0038B1F30039A1F3A82F39
:20014000E6E00C94CD020E94C802C801A22F0091A900000F02B904EC06BFB9DF003A21F4C4
:2001600006B7006806BFB3DF083A11F0003B79F4B0E001C0B395BA1750F40B2F10E0FC0143
:20018000E00FF11F0081AADF083BA1F3BA2FE4E00C94CF020A930FB700000FBF09911895E9
:2001A000479A8A9A929801B3086F01BB02B3077002BBD798DF98D698DE988898909A07B372
:2001C000007E07BB08B3007E08BB89989198089520E10AB307600ABB0AB308630ABB04B36E
:2001E0000C6104BB04B3006E04BB0BB3087F30E0F901EC5AFF4F1491012B0BBB0BB3077C34
:2002000030E0F901EB59FF4F1491012B0BBB05B3037E30E0F901EA58FF4F1491012B05BB47
:2002200005B30F7130E0F901E957FF4F1491012B05BB2A9506E00A95F1F700C02223A9F68D
:200240000BB3087F0BBB0BB3077C0BBB05B3037E05BB05B30F7105BB0895053040F51BB3C6
:20026000187F202F30E0F901E856FF4F2491122B1BBB1BB3177C202F30E0F901E356FF4FF9
:200280002491122B1BBB15B3137E202F30E0F901EE55FF4F2491122B15BB15B31F71202FEA
:2002A00030E0F901E955FF4F0491102B15BB07EE13E001501040E9F700C000000BB3087F9A
:2002C0000BBB0BB3077C0BBB05B3037E05BB05B30F7105BB0895202F00E01AB3187F1ABB5B
:2002E0001AB3177C1ABB14B3137E14BB14B31F7114BB1AEF00001A95E9F719B3177069B375
:20030000687353B35C7143B3407EE3EFF1E0E150F040E9F700C0000039B33770311741F4C7
:2003200030E0F901E856FF4F3491131709F4016019B31873161741F430E0F901E356FF4F90
:200340001491611709F4026013B31C71151741F430E0F901EE55FF4F1491511709F4046064
:2003600013B3107E141741F430E0F901E955FF4F1491411709F40860089522970FEF0983F1
:2003800007EA11E601501040E9F700C00000819963C0CE9B5EC001E20A95F1F70000CE9B9D
:2003A00058C0929A0BED15E001501040E9F700C000000EDF21E08E010E9482000881083069
:2003C00008F047C0088110E0F801E056FF4F00810093AC000091AC0040DF0091AC007BDF75
:2003E000809B0FE00F3029F521E08E010E94A30000E006BF09E910E101501040E9F700C0F8
:20040000000092984091AC004D5F01E010E00E94C30212B3102B12BB0FE714E82EE1015032
:2004200010402040E1F700C0000002B3077002BB90C021E08E010F5F1F4F0E94A30000E0AA
:2004400006BF01EB1CE001501040E9F700C000009298819B9ECF7DC006B300950F7100935D
:20046000AB000091AB00015049F00A9559F0025069F0045079F0085089F014C000E00093A3
:20048000AC0013C001E00093AC000FC002E00093AC000BC003E00093AC0007C004E00093A2
:2004A000AC0003C004E00093AC00000003EC19E001501040E9F700C00000CF9B4AC007EA1C
:2004C00011E601501040E9F700C00000CF9B41C0929A0BED15E001501040E9F700C000001F
:2004E00077DE03EF11E001501040E9F700C000000091AC00B2DE0091AC00EDDE809B0FE0A4
:200500000F30F9F403E911E101501040E9F700C0000092984091AC004D5F01E010E00E94CA
:20052000C30212B3102B12BB0FE714E82EE1015010402040E1F700C0000002B3077002BBA6
:2005400008C003E619E101501040E9F700C00000929800002296089500008895FECF0FE94E
:200560000DBF00E00EBFC0E8D0E00E94D802002311F00E94E8020E9456000E94AC020C9496
:20058000AC02000F111F4A95E2F708955A924A92BA93AA939A938A9308955D804C80BB81FB
:2005A000AA8199818881F0E0EC0FFD1FEF01089501E0089520E006D0E9F70895259102D020
:2005C000E9F708952D9301501040202F212B089584E096E0FC0105911491FC013296A591F8
:2005E000B491FC01349625913491422F432B19F0F901E4DF01C0DEDF069616E08031910776
:2006000048F308950800A00010060500A80000000404040302010004000000000000000081
:200620000000000000000000000000000000000000000000000000000000000000000000BA
:2006400000000000000000000000000000000000000000000000000000000000000000009A
:2006600000000000000000000000000000000000000000000000000000000000000000007A
:2006800000000000000000000000000000000000000000000000000000000000000000005A
:00000001FF
